:020000040800F2
:10000000F01C0020A1010008990C00085D02000806
:10001000950C000817020008D90E00080000000027
:100020000000000000000000000000009F0C00081D
:100030005B020008000000009D0C0008A10C0008F5
:10004000BB010008BB010008BB010008BB010008A0
:10005000BB010008BB010008BB010008BB01000890
:10006000BB010008BB010008BB010008BB01000880
:10007000BB010008BB010008BB010008BB01000870
:10008000BB010008BB0100080D020008BB0100080D
:10009000BB010008BB010008BB010008BB01000850
:1000A000BB010008BB010008BB010008BB01000840
:1000B000BB010008BB010008BB010008BB01000830
:1000C000BB010008BB010008BB010008BB01000820
:1000D000BB010008BB010008BB010008BB01000810
:1000E000BB010008BB010008BB010008BB01000800
:1000F000BB010008BB010008BB010008BB010008F0
:10010000BB010008BB010008BB010008BB010008DF
:10011000BB010008BB010008F10D0008BB0100088D
:1001200051020008BB010008BB010008BB01000828
:10013000BB010008BB010008BB010008BB010008AF
:10014000BB010008BB010008BB010008BB0100089F
:10015000BB010008BB010008BB010008BB0100088F
:10016000BB010008BB010008BB010008BB0100087F
:10017000BB010008BB010008BB0100080000000033
:10018000BB010008BB010008DFF810D000F02CF81C
:1001900000480047C1150008AFF30080F01C0020A4
:1001A0000648804706480047FEE7FEE7FEE7FEE711
:1001B000FEE7FEE7FEE7FEE7FEE7FEE7DD0D0008EF
:1001C00089010008D2B201E000F8012B491EFBD2E0
:1001D00070470022F6E710B513460A460446194652
:1001E000FFF7F0FF204610BD064C074D06E0E06823
:1001F00040F0010394E8070098471034AC42F6D36E
:10020000FFF7C6FFE01800081019000810B500201D
:1002100000F0CAFE10BD00BFFEE7000030B5024688
:100220000B4600BF7AB90220084C616920EA01043C
:1002300001EA000544EA0544044DAC6100BF01E059
:1002400000BF00BFFCE700BF012030BD001002402E
:1002500010B5002000F07CFE10BD704700BFFEE727
:100260002DE9F04105460C460026606800B100BF4C
:10027000134800F04FF80746124800F04BF80743C8
:10028000114800F047F80743AFB9606860B1D4E99E
:1002900000010843A1680843E168084369680B4A04
:1002A00011400843686007E0686808490840216811
:1002B0000843686000E001263046BDE8F081000098
:1002C000002001400021014000220140E010FCFF1D
:1002D000816821F0010181607047000070B504461B
:1002E0000D460026204600F015F870B9A968286868
:1002F00008436168064A114008436060A06820F422
:10030000006069680843A06000E00126304670BDC7
:10031000FFFEFFFC0146886800F001007047000006
:1003200070B504460D460026686800B100BF20463F
:10033000FFF7F0FF00BB686830B1606820F46840E8
:10034000A9680843606003E0606820F4684060606A
:10035000286800F07060E968084329690843A168CB
:10036000074A11400843A0606868E16A21F47001FF
:100370000143E16200BF00E00126304670BD00008D
:10038000FDFCFFC070B501F440744FF4407595FA60
:10039000A5F5B5FA85F5EC4000F12C0505EB8403D5
:1003A0001C6801F01F061F25B540AC4302F01F0575
:1003B00001F01F06B5402C431C6070BD70B501F004
:1003C00000744FF0007595FAA5F5B5FA85F5EC4087
:1003D00000F10C0505EB84031C6801F0F8754FF083
:1003E000F87696FAA6F6B6FA86F6F5400726AE40F7
:1003F000B44301F0F8754FF0F87696FAA6F6B6FA1F
:1004000086F6F54002FA05F52C431C6070BD426883
:1004100022F440020A4342607047426822F44002DC
:100420000A4342607047000008B505490968014366
:10043000034A1160114609680140009100BF08BDE0
:1004400030380240F0B502460B46002400211868FF
:1004500090FAA0F0B0FA80F48AE00125A54018686F
:1004600000EA050100297DD05868012802D05868AB
:1004700002281CD19868956891FAA1F6B6FA86F61A
:1004800077000326BE40B54391FAA1F6B6FA86F688
:10049000760000FA06F63543956000BFD8685568C7
:1004A0008D4301FB00F63543556000BF00BF18695E
:1004B000D56891FAA1F6B6FA86F677000326BE4013
:1004C000B54391FAA1F6B6FA86F6760000FA06F67A
:1004D0003543D56000BF5868022831D191FAA1F0A8
:1004E000B0FA80F0082814D25869156A91FAA1F67A
:1004F000B6FA86F6B7000F26BE40B54391FAA1F6CC
:10050000B6FA86F6B60000FA06F63543156200BF65
:1005100016E05869556A0E0A96FAA6F6B6FA86F6F5
:10052000B7000F26BE40B5430E0A96FAA6F6B6FAF5
:1005300086F6B60000FA06F63543556200BF00BFE6
:100540005868156891FAA1F6B6FA86F67700032680
:10055000BE40B54391FAA1F6B6FA86F6760000FAE7
:1005600006F600E003E03543156000BF00BF641CE1
:100570001868E04000287FF470AFF0BD10B5426904
:1005800021EA020302EA010443EA0443836110BD45
:1005900002480068401C0149086070474C00002078
:1005A0004FF47A71B0FBF1F2521E4FF0E0235A6122
:1005B00000229A6105221A6100BF70470149086054
:1005C000704700000000002010B5024613682C4858
:1005D00082420ED0B2F1804F0BD02A48824208D01E
:1005E0002948824205D02948824202D028488242C6
:1005F00004D123F070004C6840EA04032048824292
:1006000020D0B2F1804F1DD01E4882421AD01E4821
:10061000824217D01D48824214D01D48824211D018
:100620001C4882420ED01C4882420BD01B4882429A
:1006300008D01B48824205D01A48824202D01A488C
:10064000824204D123F44070CC6840EA0403136072
:100650008868D06200BF0888906200BF0848824264
:1006600002D00B48824203D10869106300BF00BF6B
:1006700000BF506940F00100506100BF002010BD74
:10068000000001400004004000080040000C004051
:100690000004014000400140004401400048014086
:1006A00000180040001C004000200040014608697E
:1006B00000F00100704708B54FF0E0210969009192
:1006C00000BF411C01B1401C06E04FF0E021096968
:1006D00001F4803101B1401E0028F6D108BD0000B0
:1006E0002DE9F0418EB000200B900C900D9014215C
:1006F00006A8FFF76EFD002002900390049005907D
:100700004FF48070874909680143864A1160114699
:1007100009680140019100BF00BF834800210A46DB
:10072000824B5B5CC35823F0606313437F4C645C73
:10073000035100BF00BF7D4B5B5CC35823F0C00377
:1007400013437A4C645C035100BF00BF774B5B5C82
:10075000C35823F440331343744C645C035100BF0B
:100760008215724B5B5CC35823F4907313436F4C38
:10077000645C035100BF0A466C4B5B5CC35823F4B6
:1007800000731343694C645C035100BF0215674B4F
:100790005B5CC35823F480631343644C645C035173
:1007A00000BFC214614B5B5CC35823F4C0531343B6
:1007B0005E4C645C035100BF92005C4B5B5CC358B1
:1007C00023F4C0431343594C645C035100BF00BF82
:1007D000564A525C0244526922F00402534B5B5C5D
:1007E00003445A6100BF1221514B1B68C3F302201E
:1007F000002425460346C3F1070CBCF1040F02D9BF
:100800004FF0040C01E0C3F1070C674603F1040C40
:10081000BCF1070F02D24FF0000C01E0A3F1030C72
:1008200066464FF0010C0CFA07FCACF1010C0CEA27
:10083000040C0CFA06FC4FF0010808FA06F8A8F1BF
:10084000010808EA05084CEA080200BF002904DB99
:100850001007030E3748435407E01007040E3448CE
:100860000C3001F00F031B1FC45400BF12200028DE
:1008700009DB00F01F02012191404209920002F1C0
:10088000E022C2F8001100BF00200B900C904FF442
:1008900080700D900BA92848FFF720FD00200690DE
:1008A0004FF48010079000200890022009904FF428
:1008B00040700A9006A92048FFF732FD00201E492B
:1008C000896821F4806101431B4A916000BF4FF4A5
:1008D000803002900020039002A91848FFF7C0FC66
:1008E000174A4FF400711448FFF74CFD02221449D7
:1008F0001148FFF763FD4FF400011048FFF787FD33
:10090000104A910D0C48FFF73DFD02220D490A489F
:10091000FFF754FD4FF400010848FFF778FD0EB0D3
:10092000BDE8F081443802400064024058180008D5
:100930000CED00E000E400E0002001400023014055
:1009400010002081110050812DE9F8414FF4800002
:100950002E49096801432D4A11601146096801407A
:10096000009100BF00BF3821294B1B68C3F3022050
:10097000002425460346C3F1070CBCF1040F02D93D
:100980004FF0040C01E0C3F1070C674603F1040CBF
:10099000BCF1070F02D24FF0000C01E0A3F1030CF1
:1009A00066464FF0010C0CFA07FCACF1010C0CEAA6
:1009B000040C0CFA06FC4FF0010808FA06F8A8F13E
:1009C000010808EA05084CEA080200BF002904DB18
:1009D0001007030E0F48435407E01007040E0C489D
:1009E0000C3001F00F031B1FC45400BF3820002837
:1009F00009DB00F01F02012191404209920002F13F
:100A0000E022C2F8001100BFBDE8F8813038024092
:100A10000CED00E000E400E000B587B0182101A86B
:100A2000FFF7D7FB1020FFF7FFFC4FF48070FFF7B4
:100A3000FBFC0420FFF7F8FC2020FFF7F5FC8020EA
:100A4000FFF7F2FC0120FFF7EFFC0220FFF7ECFCC0
:100A50004020FFF7E9FC0820FFF7E6FC03203A49B5
:100A6000886100BF4FF6FC700190032002900020C7
:100A7000059001A93448FFF7E5FC40F6FF700190AE
:100A8000032002900020059001A93048FFF7DAFC0E
:100A900043F6FF700190032002900020059001A909
:100AA0002B48FFF7CFFC4FF6FF7001900320029018
:100AB0000020059001A92748FFF7C4FC49F6FF7004
:100AC0000190032002900020059001A92248FFF721
:100AD000B9FC4FF6FC7001900320029000200590B5
:100AE00001A91E48FFF7AEFC4FF6FF7001900320EE
:100AF00002900020059001A91948FFF7A3FC4FF6CA
:100B0000FF700190032002900020059001A9154874
:100B1000FFF798FC4FF6FF70019003200290002031
:100B2000059001A91048FFF78DFC032001900120DA
:100B300002900220039000200490059001A9024831
:100B4000FFF780FC07B000BD00100240002002400B
:100B5000000802400014024000000240001C024055
:100B60000004024000180240000C02402DE9F04150
:100B700086B0142101A8FFF72CFB10204149096819
:100B80000143404A1160114609680140009100BFCD
:100B900000BF36213C4B1B68C3F30220062400250E
:100BA0000346C3F1070CBCF1040F02D94FF0040C4B
:100BB00001E0C3F1070C674603F1040CBCF1070F19
:100BC00002D24FF0000C01E0A3F1030C66464FF097
:100BD000010C0CFA07FCACF1010C0CEA040C0CFA49
:100BE00006FC4FF0010808FA06F8A8F1010808EA27
:100BF00005084CEA080200BF002904DB1007030EB9
:100C00002248435407E01007040E1F480C3001F03F
:100C10000F031B1FC45400BF3620002809DB00F05F
:100C20001F02012191404209920002F1E022C2F824
:100C3000001100BF44F29F10ADF8040000200290A4
:100C40006320039001A91248FFF7BEFC00BF1048C3
:100C5000006820F080000E49086000BF002049684D
:100C600021F0700101430A4A516000BF00BF1046E5
:100C7000806820F080001146886000BF06B0BDE8A3
:100C8000F0810000403802400CED00E000E400E09C
:100C90000010004000BFFEE700BFFEE7704770474E
:100CA0007047000070B505204749096821F0070129
:100CB0000143454A116000BF00BF00BF42480068C1
:100CC00000F007000528F8D14FF480403F4909683B
:100CD00021F4804101433D4A116000BF00BF3C4800
:100CE000006840F480303A49086000BF00BF00BF90
:100CF00037480068C0F340400028F8D04FF4800027
:100D00000421A822002340EA010444EA8214304D61
:100D10002D1D2D682F4E35402C432D4D2D1D2C6043
:100D20002C46246824F440341C432C6000BF00BFD0
:100D3000281F006840F08070291F086000BF00BFB6
:100D400000BF23480068C0F340600028F8D000BF0F
:100D500000BF1E484068C0F380300028F8D0002053
:100D60001B490831096821F0F0010143184A083293
:100D7000116000BF4FF4A0501146096821F4E05102
:100D80000143116000BF4FF400401146096821F48F
:100D900060410143116000BF02201146096821F043
:100DA00003010143116000BF00BF00BF08480830C5
:100DB000006800F00C000828F7D10748FFF7F0FBA7
:100DC0000548FFF7FBFB70BD003C0240007000408F
:100DD000003802400080BFFF007A030A0348006821
:100DE00040F47000014908607047000088ED00E0A1
:100DF00010B53748FFF75AFC012868D100BF00BF83
:100E000033480069C0F3400060B100BF3048C0689B
:100E1000C0F3400030B100BF6FF002002C49086100
:100E200000BF00BF00BF2A480069C0F3800060B166
:100E300000BF2748C068C0F3800030B100BF6FF02A
:100E400004002349086100BF00BF00BF20480069BB
:100E5000C0F3C00060B100BF1D48C068C0F3C0004F
:100E600030B100BF6FF008001949086100BF00BF32
:100E700000BF17480069C0F3001060B100BF1448FC
:100E8000C068C0F3001030B100BF6FF0100010490F
:100E9000086100BF00BF0E48FFF708FC01280CD115
:100EA00000BF0B48C06800F0010030B100BF6FF018
:100EB00001000749086100BF00BF00BFFFF768FBE2
:100EC00000BF04480068401C0249086000BF10BD14
:100ED000001000404400002000BFFEE702E008C808
:100EE000121F08C1002AFAD170477047002001E0A4
:100EF00001C1121F002AFBD170470000014601F119
:100F0000100000E0001D02681AB9024A12689042FF
:100F1000F8D370472400002010B50648046803E0A9
:100F20002046FFF7EBFF0446034800688442F7D3EE
:100F300010BD0000200000202400002010B501E0BA
:100F400000F8011B131EA2F10104A2B2F8D110BDDA
:100F500070B5054605EBC500124901EB80040CB1E4
:100F6000012100E00021084640F22911FFF756F95F
:100F700060680168C1F3C02139B160684FF4006155
:100F8000816000BF2068FFF7A3F960680168C1F3C2
:100F9000402129B160684FF40071816000BF00BF3B
:100FA00070BD00008018002070B5054605EBC50037
:100FB0000D4901EB80040CB1012100E0002108463D
:100FC0004FF4A071FFF72AF920680168C1F34011BE
:100FD00041B16069401C606120686FF020010160D0
:100FE00000BF00BF70BD0000801800200146002037
:100FF00001F001020AB1421CD0B201F002020AB1B2
:10100000421CD0B201F004020AB1421CD0B201F07D
:1010100008020AB1421CD0B201F010020AB1421C0F
:10102000D0B201F020020AB1421CD0B201F040025D
:101030000AB1421CD0B201F080020AB1421CD0B207
:1010400001F480720AB1421CD0B201F400720AB1FC
:10105000421CD0B201F480620AB1421CD0B201F449
:1010600000620AB1421CD0B201F480520AB1421CA3
:10107000D0B201F400520AB1421CD0B201F4804255
:101080000AB1421CD0B201F400420AB1421CD0B2F3
:1010900001F480320AB1421CD0B201F400220AB13C
:1010A000421CD0B201F480220AB1421CD0B201F439
:1010B00000320AB1421CD0B2704700002DE9FF4F48
:1010C00081B006460F469046DDE90F95032E01DA02
:1010D000012100E0002108461C21FFF79FF80FB115
:1010E000012100E0002108461D21FFF797F8B8F123
:1010F000000F01D0012100E0002108461E21FFF76A
:101100008DF8B9F1000F01DD012100E00021084652
:101110001F21FFF783F806EBC600744901EB80043A
:10112000242200212046FFF709FF2760C4F804802D
:101130000498A0600E98E0602561A4F818902846F5
:10114000FFF754FFA076A07E00FB09F0A083A08BE0
:101150004FEA400A5146012000F060FB2062216AFC
:1011600009B1012100E0002108463221FFF756F8BD
:10117000A18B49040A0C0021206AFFF7DFFE201D25
:1011800007C85B4B5B5CC35823F060631343DFF815
:1011900060C11CF801C040F80C3000BF554AD4E9CA
:1011A0000101534B5B5CC358DFF84CC103EA0C03ED
:1011B0001343DFF83CC11CF801C040F80C3000BFFD
:1011C0004FF0000BD4E900A0A1684FF0000ECDF85D
:1011D00000E0BBF1000F04D10AF14C0ECDF800E0A5
:1011E00003E0DFF818E1CDF800E0009AD4E901ABA4
:1011F000236ADFF8FCE01EF80BE05AF80EE00EF070
:10120000C00C00BFBCF1400F0ED1DFF8E4A01AF80B
:1012100001A08244CAF80C20DFF8D4A01AF801A07B
:101220008244CAF808300DE0DFF8C4A01AF801A023
:101230008244CAF80820DFF8B8A01AF801A0824456
:10124000CAF80C3000BFA28BD4E90101284B5B5CCB
:1012500003445B686FF30F031343DFF894C01CF87B
:1012600001C08444CCF8043000BFD4E90101204A15
:10127000525C825842F001021D4B5B5CC25000BFC1
:1012800002212068826822F002020A43826000BFC5
:101290004FF440712068826822F440720A438260F1
:1012A00000BF05F4002028B14FF4000113480838AE
:1012B000FFF7B3F805F4003028B14FF400010F48F0
:1012C0000838FFF7AAF80A20FFF7F5F920688168C7
:1012D00041F00101816000BF2068816841F08041D8
:1012E000816000BF05B0BDE8F08F000080180020CD
:1012F000B4180008002D02001F80FCFF08230140E5
:101300002DE9F04705468846032D01DA012100E06A
:1013100000210846EE21FEF781FF4FF0000900266C
:1013200005EBC500104901EB80040CB1012100E080
:1013300000210846F221FEF771FF206A00EB480702
:10134000002006E039880E44411C88B2A17E07EBDC
:101350004107218B8142F5DC208BB6FBF0F01FFAB0
:1013600080F94846BDE8F087801800200C4B1988AA
:101370009B1C1A88431A00EE903AF8EEE01A531AB2
:1013800000EE903AF8EEE00A81EEA01ADFED051AC1
:10139000F3EE0E0A41EE210AB0EE600A704700003B
:1013A0002C7AFF1F0000A0420E49098840F6E44253
:1013B000514340F6FF72B1FBF2F100EE101AB8EEA5
:1013C000400AF0EE400A00EE100AB8EE400A80EE45
:1013D000801A9FED050A21EE001ADFED041A81EE56
:1013E000210A70472A7AFF1F00F07F4500007A44E7
:1013F00000200B4908600B49086000BF00BF0A4885
:10140000006840F001000849086000BF00BF0846BE
:10141000C06840F00100C86000BF00BF7047000016
:1014200008000020100000200010004010B5034804
:1014300000F01CF8024800F087F810BD08000020FA
:10144000100000200EB54FF420204FF4C871002288
:101450001346CDE900210290024A03490020FFF71C
:101460002DFE0EBD006402400020014038B5044648
:1014700000200090206810B112281DD112E000BF9A
:1014800000F02AF80F4880ED000A00F041F80D48FE
:1014900080ED010A00BF0C480068606000BF1220A8
:1014A000206000BF084960680968081A642801D2F2
:1014B000002038BD00BFE3E700202060009003203B
:1014C000F7E70000180000204400002001490860F0
:1014D000704700004800002010B52DED028B9FEDF5
:1014E0000A0AB0EE408A00210846FFF709FF0749C3
:1014F00008800888FFF73AFFB0EE408AB0EE480A4D
:10150000BDEC028B10BD00000000000004000020B4
:1015100010B52DED028B9FED0A0AB0EE408A012135
:101520000020FFF7EDFE074948804888FFF73CFFA1
:10153000B0EE408AB0EE480ABDEC028B10BD000050
:10154000000000000400002038B504460020009090
:10155000206810B1252816D10BE000BF012000F053
:1015600019F800BF0A480068606000BF25202060AD
:1015700000BF074960680968081A642801D2002082
:1015800038BD00BFEAE70020206000900320F7E7A5
:101590004400002010B5044614B1012C0AD104E027
:1015A00001210648FEF7EAFF05E002210348FEF7A5
:1015B000E5FF00E000BF00BF10BD000000100240CA
:1015C00008B54FF48040444909680143424A11601C
:1015D000114609680140009100BF00BF8003111F40
:1015E00009680143121F116011460968014000910A
:1015F00000BF00BF03200246384B19684FF6FF03B7
:101600001940374B0B4343EA0221344B196000BFAA
:10161000011F1B68C3F302200F2400250346C3F1FA
:10162000070CBCF1040F02D94FF0040C01E0C3F128
:10163000070C674603F1040CBCF1070F02D24FF010
:10164000000C01E0A3F1030C66464FF0010C0CFA0C
:1016500007FCACF1010C0CEA040C0CFA06FC4FF090
:10166000010808FA06F8A8F1010808EA05084CEA9A
:10167000080200BF002904DB1007030E1948435479
:1016800007E01007040E15480C3001F00F031B1F74
:10169000C45400BFFFF706FB134800681349B0FBB2
:1016A000F1F084B22046FFF711FFFFF7B5F9FFF71D
:1016B0004BF9FFF75BFAFFF713F8002000F018F87A
:1016C000012000F015F8FFF7BDFEFFF791FE01E0E5
:1016D000FFF7ACFEFCE70000443802400CED00E0F0
:1016E0000000FA0500E400E00000002040420F0086
:1016F00010B504460C4951F824104A000B4951F822
:101700002400002100F09EF8094951F824200749DF
:10171000083951F82400002100F094F80121034811
:101720000830015510BD00009C180008380000204A
:10173000AC1800082DE9F04704460F460025A946DD
:101740002348005D20B922481838016820468847A0
:101750001FB94FF0FF30BDE8F0871E4850F8240055
:10176000B7FBF0F61B4850F82400B7FBF0F100FB84
:10177000117000B1761C184850F82400451E22E074
:101780001348083850F8240030F8150010B909F152
:10179000010901E04FF00009B14513D14FF00008F5
:1017A00009E00B48083850F8240005EB080220F83F
:1017B000126008F10108B045F3D3064850F8240040
:1017C0006843C8E76D1E002DDADA4FF0FF30C2E73C
:1017D00040000020A41800089C18000810B501461D
:1017E0000023002207E00B4850F8210030F81200D7
:1017F00000B15B1C521C084850F821009042F2D8FE
:1018000064205843044C54F82140B0FBF4F0C0B2BB
:1018100010BD0000380000209C18000870B5044678
:101820000E4631462046FFF785FF0546681C08B97D
:10183000002070BD024850F824002844F9E7000059
:101840003000002030B5034601E003F8011B141EF0
:10185000A2F10102F9D130BD102840587088A0B81B
:10186000000000000404040000080000000800005C
:10187000080000000800020406080A0C0001020328
:101880000405065F6C697374006C69737420616C85
:101890006C20636F6D6D616E6400000000020000DB
:1018A0000002000008000000080000000010000016
:1018B00000100000102840587088A0B800000000F8
:1018C00004040400000800000008000008000000F4
:1018D0000800020406080A0C0001020304050600C1
:1018E00010190008000000206C000000DC0E000849
:1018F0007C1900086C000020841C0000EC0E00081D
:101900007C19000800C0012000100000EC0E000847
:101910000024F400000000000000000000000000AF
:1019200000000000000000000000000000000000B7
:101930000000000000000000F1160008DD1700089C
:101940008000002000C001208010002080140020B2
:101950000000000000000000000000000000000087
:1019600000000000000000000000000083180008D4
:0C19700089180008C6E533B4190F000800
:040000050800018965
:00000001FF
